:02000000804E30
:10005000758140119974807841117274C090008844
:10006000116480FE11B2E493A3B40001221200E2F5
:1000700080F411B2E8C4540F9000889311E2E85460
:100080000F9000889311E222303132333435363705
:10009000383941424344454600743811B2740F1157
:1000A000B2740111B2740611B211EF11EF11EF1118
:1000B000EF22C2B2C2B0C2B111BFD2B0D2B12213CC
:1000C000929013929113929213929313929413928B
:1000D00095139296139297D2B200000000C2B2110B
:1000E000EF22C2B2D2B0C2B111BFC2B0D2B122C0EF
:0A00F000F075F0FFD5F0FDD0F0220E
:00000001FF
